:020000040000fa
:080000001015040000000000cf
:020000040000fa
:102a20000f4221000e7f24000e01880000000000ec
:102a30000c00070020792100010020001f00070082
:102a4000000020000000e000020032000000020050
:102a5000000000008e330200000000000040da0099
:102a60000000fe004440a900600c20000000e000cf
:102a70000300320000002000a00188004440a800ac
:102a800000000600f03fb1000180b10006003500f3
:102a9000ee03090000000000403fb1000180b100da
:102aa000fbff3d001000b000203fb00002003500e9
:102ab000008009000000000000000600910188006d
:102ac000800078000000eb0015003700e280400035
:102ad00032a0b4009101ba00e280400032a0b400fc
:102ae0009102ba00e280400032a0b4000002eb0084
:102af000472bde00f507b200602ce10004003a002d
:102b00000059eb008301e900fdff3e00040037009f
:102b10006128e100010032000082eb0004000700a0
:102b20001101ba000200e000e8ff3a0000000600d0
:102b30003159ba008301e9000c0032002159ba0072
:102b40008301e900080032000400e00003003a00bd
:102b5000e280400032a0b400f5ff370011d9ba007e
:102b60008301e900faff3a008100e800e1804000bb
:102b700032a0b40000000600839f68000100e0005e
:102b800002003d0060001000e08018000300e0003b
:102b900002003d0060011100e081190011000700f2
:102ba0004f00e00002003b0060001000e0801800d1
:102bb0000000060033c2bf000004a20061006000f4
:102bc000000006008000780030c2bf006640600050
:102bd000e64f500001003200f10fb200a111880051
:102be0000000060002025000838258006100390094
:102bf00003037100620032000503720059003200c5
:102c00000300e0005500330017003a000100e00027
:102c10004b0032000208e1000600310011000900fb
:102c20004288d800010178008001eb008000eb00b1
:102c3000000006006110e100550032000002be00f5
:102c4000110009008280d80080027800040078001a
:102c5000110009004288d800010178008001eb00d2
:102c60008500780000000600889fbe008a9fbe0095
:102c70008c9fbe000386cf000c06e9008c1f7800f5
:102c80008c19dd00f00216000512de00848171004f
:102c90000c11dd000003be008004eb00053cde00eb
:102ca0008c3bdd000532de00848373000c33dd00d5
:102cb0000700780088007800110009004388d800d8
:102cc0000202b8000306b8008c82420060854e0004
:102cd0008005eb000402530085825b000a055c005e
:102ce0008b855c000b0033008000eb004f06780002
:102cf0000c21de00700516000a2ddd000a017100ae
:102d00008c29de004f06be004f05be004f04be00fa
:102d1000000006000202420083824a0060054d0066
:102d2000e0854d000000e9000b00e000eeff3d00f3
:102d30000202420083824a000000e900eaff3700f5
:102d40000000e00012003200110009000280d800eb
:102d5000010178008000eb00000006000401be00c5
:102d6000010037006011b800100020008000eb0067
:102d7000000006000001be006000b8000000060070
:102d80000001be00f0ff2f00f1ff2f000000060041
:082d90006011b800000006000c
:020000040000fa
:020000040005f5
:0457f800be430000ac
:020000040000fa
:020000040005f5
:0457fc00e13e00008a
:020000040000fa
:102800001015040000000000e017040000000000a4
:10281000e017040000000000e017040000000000c2
:10282000e017040000000000e017040000000000b2
:10283000e017040000000000e017040000000000a2
:10284000e0170400000000007630040000000000e3
:10285000e017040000000000e01704000000000082
:102860003632040000000000e01704000000000001
:10287000e017040000000000e01704000000000062
:10288000e017040000000000e01704000000000052
:10289000e017040000000000e01704000000000042
:1028a000e017040000000000e01704000000000032
:1028b0004c32040000000000e0170400000000009b
:1028c000e017040000000000e01704000000000012
:1028d000e017040000000000e01704000000000002
:1028e000e017040000000000e017040000000000f2
:1028f000e0170400000000000630040000000000a3
:102900000030040000000000e01704000000000098
:10291000e017040000000000e017040000000000c1
:10292000e017040000000000e017040000000000b1
:10293000e017040000000000e017040000000000a1
:10294000e017040000000000e01704000000000091
:10295000e017040000000000e01704000000000081
:10296000e017040000000000e01704000000000071
:10297000e017040000000000e01704000000000061
:10298000e017040000000000e01704000000000051
:10299000e017040000000000e01704000000000041
:1029a000e017040000000000e01704000000000031
:1029b000e017040000000000e01704000000000021
:1029c000e017040000000000e01704000000000011
:1029d000e017040000000000e01704000000000001
:1029e000e017040000000000e017040000000000f1
:1029f000e017040000000000e017040000000000e1
:102a0000e017040000000000e017040000000000d0
:102a1000e017040000000000e017040000000000c0
:020000040000fa
:1000080004140000081400000c1400001014000070
:10001800141400000c1500000c1500000c1500004d
:10002800181400001c140000201400002414000000
:100038000c150000281400002c14000030140000d7
:1000480034140000381400003c1400004014000070
:1000580044140000481400000c1500000c150000a2
:100068004c140000501400005414000058140000f0
:100078005c1400000c1500006014000064140000fb
:100088000c150000681400006c14000070140000c7
:1000980074140000781400007c1400008014000020
:1000a80084140000881400000c1500000c150000d2
:1000b8000c1500008c14000090140000941400002b
:1000c800981400009c140000a0140000a414000060
:1000d800a8140000ac1400000c1500000c1500005a
:1000e8000c150000b0140000b41400000c1500003a
:1000f8000c150000b8140000bc1400000c1500001a
:100108000c1500000c1500000c1500000c15000063
:100118000c1500000c150000c01400000c150000a0
:100128000c150000c4140000c8140000cc14000012
:100138000c1500000c1500000c1500000c15000033
:10014800d01400000c1500000c1500000c15000060
:100158000c150000d41400000c1500000c1500004c
:100168000c150000d8140000dc140000e014000096
:10017800e4140000e8140000ec140000f01400007f
:10018800f4140000f8140000fc140000001500002e
:1001980004150000081500000c1500000c150000df
:1001a8000c1500000c1500000c1500000c150000c3
:1001b8000c1500000c1500000c1500000c150000b3
:1001c8000c1500000c1500000c1500000c150000a3
:1001d8000c1500000c1500000c1500000c15000093
:1001e8000c1500000c1500000c1500000c15000083
:0801f8000c1500000c150000bd
:020000040000fa
:102d9800120100000002000000000000000800000e
:102da800d80400003f0000000200000001020000fb
:102db80000010000090200002900000001010000d4
:102dc80000c00000320900000400000000020000fa
:102dd80003000000000000000921000011010000ac
:102de80000010000221c000000070000058100000f
:102df8000340000000010000070500000103000077
:102e08004000000001000000040300000904000065
:102e1800340300004d00000069000000630000005a
:102e2800720000006f0000006300000068000000ee
:102e3800690000007000000020000000540000003d
:102e48006500000063000000680000006e000000dc
:102e58006f0000006c0000006f00000067000000b9
:102e68007900000020000000490000006e0000000a
:102e7800630000002e0000002e0300005300000035
:102e8800690000006d000000700000006c00000088
:102e98006500000020000000480000004900000014
:102ea800440000002000000044000000650000000d
:102eb8007600000069000000630000006500000063
:102ec8002000000044000000650000006d000000c4
:102ed8006f00000006000000ff09000001a10000cb
:102ee800011900000129000040150000012500001b
:102ef800407500000895000040810000001900009e
:102f0800012900004091000000c00000de9600008a
:0c2f1800089700000c9700004097000094
:020000040000fa
:106000000000fa000080fa0000400600809fbe00f9
:10601000821f78000000fa0087c0a90032c2bf00ca
:10602000614060000004e000fcff3200202f2100ee
:10603000104078000081fb00b011800080407800a3
:106040002092200001717800202f2100104078005c
:106050000081fb00202f2100104078008080fb0091
:1060600020922000e14078006098200001717800c3
:10607000202f2100104078008040e800202f2100d0
:1060800001487800202f2100104078008080fb001c
:10609000102f2100104078000080fb000000e90074
:1060a000808f500003003a00212f21000040eb00b8
:1060b00080487800202f2100104078008080fb006d
:1060c0002092200061407800ea4f500003003a001f
:1060d000212f21000040eb00804878000080fa006a
:1060e0004f0178004f00be00004006003600f80067
:1060f000809fbe00829fbe00849fbe00869fbe0020
:106100000400fa00602f2100104078008040e80071
:10611000602f210001487800602f21001040780096
:10612000e34f5000c9003a00612f21000040eb000e
:1061300080487800e2c2bf00614060000004e000d7
:1061400061003a00402f2100104078000004e00078
:106150005d003200d8030700c3030700402f210071
:1061600010407800e14f500054003a00e0a42000b5
:10617000104078000080fb001007980010032000fa
:106180009e009000808f50000e003200100320000f
:106190009e009000808f500005003c00000320000e
:1061a0009e009000808f50000a00320046003700a9
:1061b000900320009e009000808f500042003c0021
:1061c00004003700d130210080c0b300804878003f
:1061d0003d003700cae2a90000000000ca62a90021
:1061e00000000000e0a420009040780000c3b3004d
:1061f00080cf500003003a00e1a42000a0c3b30008
:1062000080487800e0a42000104078008080fb00e7
:1062100000fd2f0000804000a0988800412f210041
:106220000040eb00804878000000eb00b098880048
:1062300013003700b3988000a0988000b2988000c7
:106240006f00b90002004000ea00400020882000f2
:106250000080400090407800e0a420008171780028
:10626000b09880000000e800b0988800402f21001e
:10627000104078008040e800402f2100014878005d
:10628000a0988000b29880006f00b9000200400022
:10629000ea00400020882000008040009040780004
:1062a00000c2b30080cf5000e2ff3a00d13021009d
:1062b00090c0b3008048780003003700d13021003f
:1062c00090c0b30080487800e2c2bf006140600027
:1062d0000004e0005b003200402f210010407800f5
:1062e000e14f500057003600730307005e030700bc
:1062f000402f210010407800e14f5000510036003f
:10630000e0a42000104078000080fb00000f78001f
:10631000100320009e007800808f5000490032005a
:10632000100320009e007800808f500005003c0084
:10633000000320009e007800808f5000050032008e
:1063400040003700900320009e007800808f5000ae
:106350003c003c00e0a420009040780000c3b30063
:1063600080cf500003003a00e1a42000a0c3b30096
:1063700080487800e0a42000104078008080fb0076
:1063800000fd2f0000804000a09888000000eb0076
:10639000b09888000c003700a0988000b298800068
:1063a0006f00b90002004000ea0040002088200091
:1063b0008080400000c2b30080487800b098800020
:1063c0000000e800b0988800b0988000ee0f500000
:1063d000f1ff360010002000b09888000f00370051
:1063e000a2988000b09880008001e900b1988000f8
:1063f000e0a42000614278006f10b9000300400063
:10640000ea00400020882000008040000448780016
:10641000b09880000000e800b0988800402f21006c
:10642000104078008080fb00b0988000808f500082
:10643000ebff3e00412f21000040eb008048780038
:10644000db07070005e1a90011e1a8008460a900ad
:106450000080fa004f03be004f02be004f01be0095
:106460004f00be003600f90000400600809fbe00cd
:106470000000fa00702f210011c0b300014878001d
:106480000000eb003008880084e0a9000080fa00da
:106490004f00be00004006003600f800809fbe009e
:1064a000829fbe00849fbe00869fbe000200fa004d
:1064b00011e1a90000102700210020004215020070
:1064c00000000000101780006f4f6000502f210067
:1064d000104078001e406800104798008660a900b0
:1064e0001e4090000080fb004300de006100600061
:1064f0000004e0000b0032001e80fb004300de00c1
:10650000610060000004e00003003200cae2a9005c
:106510000000000003003700d130210050c0b3005c
:10652000804878001e4090000080fb004200de00a2
:10653000610060000004e000120032001e80fb00d9
:106540004200de00610060000004e0000c00320048
:10655000ca62a90000000000e2c2bf006240600001
:106560000004e00007003a00a0a5200010407800d9
:106570008040e800a0a52000014878000100370015
:10658000660907001e4090000080fb000000d1005b
:10659000610060000004e000290032001e80fb0062
:1065a0000000d100610060000004e0001e00320025
:1065b000a0a52000104078000004e0001800320080
:1065c000a0a5200010407800ea4f500003003a00d8
:1065d000a1a520000040eb0080487800402f21005a
:1065e000104078000081fb00a0a52000104078003a
:1065f0000043b00080407800e0a4200001717800e2
:10660000402f2100104078008040e800402f2100fa
:1066100001487800a1a520000040eb0080487800e8
:1066200005e1a8000600370005e1a9000000eb0025
:1066300000088800612f21000040eb0080487800ae
:106640001e4090000080fb00610060000004e0003c
:1066500020003200f13021000040eb00804878003b
:106660001e80fb00610060000004e0000f003200ab
:10667000e030210010407800e24f5000040032006a
:10668000e030210010407800e44f500011003a0043
:10669000d130210070c0b30080487800412f210024
:1066a0000040eb00804878000a003700f1302100fc
:1066b00010c0b30080487800e0302100104078001e
:1066c000e34f500003003a00d130210060c0b30016
:1066d00080487800502f21001e48780000102700c5
:1066e000210020004215020000000000a0a52000ab
:1066f000104078000004e00001003a0011e1a80019
:106700000080fa004f03be004f02be004f01be00e2
:106710004f00be003600f900004006000000fa00fd
:106720003e0307001f00070000202100a1072000f2
:106730004215020000000000cae2a90000000000ab
:10674000ca62a9000000000000202100a10720006b
:1067500042150200000000007f0807000020210011
:10676000a10720004215020000000000cae2a900b3
:1067700000000000ca62a9000000000000502300d1
:10678000c100200042150200000000009660a80031
:10679000ee4702000000000019000700280507006e
:1067a000fbff37000000fa00cae2a9000000000069
:1067b000ca62a90000000000765b02000000000031
:1067c000e13621000040eb0080487800ff0607001a
:1067d0004d02070006470200000000000000000014
:1067e00010002000f097880010178000ef40600034
:1067f000502f2100014878000080fa0000000600b8
:106800000800fa00889fbe00e2c2bf00624060003c
:106810000004e00006003a00e2c2bf0061406000f0
:106820000004e00002003200ca02a800fb013700a9
:10683000ca02a900702f210010407800e14f5000db
:106840009d013a00712f21000040eb008048780044
:10685000d030210010407800e34f50000700320094
:10686000d030210090407800c030210001487800ed
:10687000d130210030c0b30080487800c030210002
:10688000104078000080fb006101b90022079800e9
:106890003307980090002000010020002e01900096
:1068a000be019000800f5100818f590062013e00af
:1068b0002e009000be00900000600100090037002b
:1068c0001c003700bf0037000d0037002d003700d7
:1068d0003c0037004b0037005f0037007200370084
:1068e00087003700ca02a90030062000809888007f
:1068f000c130210050c0b300804878004e013700fd
:106900000060fe00ca02a900809880000000e80034
:10691000809888008198800040062000808f500079
:1069200045013a00c00107000000eb008098880094
:1069300041013700c13021000040eb008048780061
:10694000a19e200020c5b30080487800b19e2000a1
:10695000c0c2b30080487800c19e200010c3b300bd
:1069600080487800d19e2000d0c0b30080487800d5
:10697000e19e20000040eb0080487800a70507005a
:106980002d0137000060fe00ca02a900c1302100bd
:1069900020c0b30080487800a19e200020c4b3002e
:1069a00080487800b19e2000d0c0b30080487800b5
:1069b000c19e20000040eb0080487800970507004a
:1069c0001d0137000060fe00c130210020c0b3006f
:1069d00080487800a19e200010c5b3008048780050
:1069e000b19e2000d0c0b30080487800c19e200036
:1069f0000040eb00804878009b01070087050700f6
:106a00000d013700ac010700a19e200030c4b30087
:106a100080487800b19e2000d0c0b3008048780044
:106a2000c19e20000040eb00804878008e010700e6
:106a30003006200080988800f130210020c0b3008b
:106a400080487800c130210030c0b3008048780011
:106a500072050700f8003700a19e200050c4b30063
:106a600080487800b19e2000d0c0b30080487800f4
:106a7000c19e20000040eb00804878007a010700aa
:106a80003006200080988800f130210020c0b3003b
:106a900080487800c130210050c0b30080487800a1
:106aa0005e050700e4003700a19e200010c4b3007b
:106ab00080487800b19e200020c5b300804878004f
:106ac000c19e2000d0c0b30080487800d19e200035
:106ad0000040eb0080487800412f21000040eb008f
:106ae000804878003006200080988800c13021005e
:106af00050c0b3008048780048050700ce0037003a
:106b0000a19e200010c4b30080487800b19e2000f0
:106b1000c0c2b300804878000000eb00a098880055
:106b20000a003700a09880000081e800a19880004a
:106b3000e0a42000e1407800a09e200001717800d0
:106b4000a09880000000e800a0988800402f210055
:106b5000104078008080fb00a0988000808f50005b
:106b6000f0ff3e00402f2100104078000080fb0025
:106b70000081e800a19e2000d0c0b30000f17800a1
:106b8000402f2100104078000080fb00630140008e
:106b9000a19e20000040eb0000f17800412f210071
:106ba0000040eb0080487800300620008098880084
:106bb000c130210050c0b30080487800170507009d
:106bc0009d0037004092200090407800b0c4b30090
:106bd00080cf500007003a0023010700c030210099
:106be00051c0b300014878000000eb0040978800d6
:106bf0009000370050922000104078000080fb0089
:106c000010079800400320009e009000808f5000e5
:106c100039003200400320001e019000800f510017
:106c200009003c00000320009e019000808f51006d
:106c300052003500200320009e009000808f5000fd
:106c40001200340023003700600320001e01900072
:106c5000800f51003a003200600320009e01900036
:106c6000808f51002d003500300420009e009000e0
:106c7000808f500032003200f00620001e0190008c
:106c8000800f5100370032003c003700e130210016
:106c90000040eb0080487800c130210050c0b300b4
:106ca00080487800509780000000e80050978800e6
:106cb00050978000e50f50005e003a00c030210080
:106cc00041c0b300014878000000eb0050978800f5
:106cd00058003700e130210010c0b3008048780030
:106ce000c130210030c0b300804878000000eb00c4
:106cf000409788004f003700e130210020c0b300ea
:106d000080487800c130210030c0b300804878004e
:106d10000000eb004097880046003700e13021007a
:106d200030c0b30080487800c130210030c0b300cb
:106d3000804878000000eb00409788003d00370055
:106d4000e130210040c0b30080487800c13021000c
:106d500030c0b300804878000000eb004097880006
:106d600034003700c03021008040eb00014878003b
:106d700030062000809888002e0037004097800061
:106d80000000e80040978800c130210050c0b300e7
:106d90008048780040978000e10f500025003400c3
:106da000e0302100104078000004e00020003a00ac
:106db000a19e200020c5b30080487800b19e20002d
:106dc000c0c2b30080487800c19e200010c3b30049
:106dd00080487800d19e2000d0c0b3008048780061
:106de000e19e20000040eb00804878008b04070003
:106df00000202100a1072000421502000000000031
:106e000000202100a1072000421502000000000020
:106e100000202100a1072000421502000000000010
:106e200000202100a1072000421502000000000000
:106e30000000fe008c00070067a0a8009660a80074
:106e4000e030210010407800e44f50000b003a0081
:106e5000e2c2bf00614060000004e00007003200b1
:106e6000f0302100104078000004e00003003a00f8
:106e7000c130210070c0b30080487800e0302100ac
:106e800010407800e34f50000b003a00e2c2bf0010
:106e9000614060000004e00007003a00f03021008b
:106ea00010407800e14f500003003a00c13021004b
:106eb00060c0b30080487800e030210010407800c6
:106ec000e34f50000a003a00e2c2bf006140600098
:106ed0000004e000060032001300200002fa200047
:106ee000514d2100100020009704070005003700d5
:106ef0008001eb000001eb008000eb000000eb00e4
:106f0000650407000e0078001a0707001e007800cd
:106f10000097880043988000002e210010407800e0
:106f20008080fb00102e2100104078000080fb00c4
:106f30004800dd00008040000001780083804100af
:106f4000c0a5200000804000020878004098800022
:106f50000000e8004098880041988000f00320007d
:106f6000808f5000020036000000eb00409888003f
:106f70000000eb00e05688000000eb00a0988800bd
:106f80000b003700a098800080004000c0a52000c2
:106f90000080400090007800e056800000804000b3
:106fa000e0568800a09880000000e800a0988800c3
:106fb000a1988000f0032000808f5000f1ff360080
:106fc000e05680004600de00e0568800e056800073
:106fd0006104b800264480003744800088007800af
:106fe00006007800000ab80007c0b9000501780063
:106ff0000001410009b0b90000014100820278009f
:10700000c129dd004f20de0000807100cf28de00a6
:10701000f05688000000eb00509888004f04be0036
:107020000080fa00000006000000fa00c1302100d4
:1070300020c0b30080487800a19e200010c5b30096
:1070400080487800b19e2000d0c0b300804878000e
:10705000c19e20000040eb0080487800ef0307004d
:107060000080fa00000006000000fa00202f210036
:107070008040eb00014878000000eb00a0988800f9
:1070800007003700a29880002192200000c2b300c0
:1070900000f17800a09880000000e800a098880027
:1070a000a198800030062000808f5000f5ff360048
:1070b0000080fa00000006000000fa00302f2100d6
:1070c0008040eb00014878000000eb00a0988800a9
:1070d00007003700a2988000a19e200000c2b300e4
:1070e00000f17800a09880000000e800a0988800d7
:1070f000a198800030062000808f5000f5ff3600f8
:107100000080fa00000006000000fa00881f7800e6
:10711000e0568000504488000000eb00a0988800f2
:1071200015003700a8988000e0568000010020007c
:10713000470add00c902de00850272004702dd0059
:10714000a09880000000e8006101b8000400be00c3
:10715000bc15020000000000000178008800440017
:1071600000ae20000080400002087800a098800057
:107170000000e800a0988800a1988000f03f20005f
:10718000808f5000e7ff36004f0478000080fa003f
:10719000000006000600fa00000f780011079800b2
:1071a000220798001e0090009e0f100002003d0074
:1071b0001e009000000f78002e0090009e0f10001f
:1071c000020034002e009000000f78001e007800ae
:1071d0000080fa00000006000c00fa00008fbe00dc
:1071e0002207980033079800440798005507980035
:1071f0002e009000be009000be0f1000ae8f180051
:1072000003003d002e009000be009000008fbe00e5
:107210004e009000de009000be0f1000ae8f1800f0
:10722000030034004e009000de009000008fbe008e
:107230001e00be000080fa00000006000400fa00f4
:10724000000f7800214798001e00e00008003d0074
:107250001e0fea002e4090008080fb001e00780088
:107260000180de00000f78001e0fea0005003700e5
:107270002e4090008080fb001e0078000180de0020
:10728000000f78001e0078000080fa000000060061
:107290000600fa00008fbe00424798001e00be00a4
:1072a000e00f5000e08f580013003d001e00be00ac
:1072b00060001000e0801800008fbe004e4090007b
:1072c0000081fb001e00be00820178008301e900fe
:1072d000030033008180d1000080d300fbff370022
:1072e000008fbe001e00be0060001000e08018008d
:1072f000008fbe000a0037004e4090000081fb0066
:107300001e00be00820178008301e9000300330003
:107310008180d1000080d300fbff3700008fbe00ca
:107320001e00be000080fa00000006000400fa0003
:10733000000f7800214798001e00e00008003d0083
:107340001e0fea002e4090008080fb001e00780097
:107350000100dd00000f78001e0fea000500370075
:107360002e4090008080fb001e0078000100dd00b0
:10737000000f78001e0078000080fa000000060070
:107380000600fa00008fbe00424798001e00be00b3
:10739000e00f5000e08f580013003d001e00be00bb
:1073a00060001000e0801800008fbe004e4090008a
:1073b0000081fb001e00be00820178008301e9000d
:1073c000030033000000400081804800fbff3700cd
:1073d000008fbe001e00be0060001000e08018009c
:1073e000008fbe000a0037004e4090000081fb0075
:1073f0001e00be00820178008301e9000300330013
:107400000000400081804800fbff3700008fbe0075
:107410001e00be000080fa00000006000000fa0016
:107420004007a9000080eb0060198800dea2a800d8
:10743000de82a800de62a800de42a800de22a800ec
:10744000de02a800df62a800df42a800df22a80059
:10745000d8a2a900d882a900d862a900d842a90060
:10746000d822a900d802a900d962a900d942a9004e
:10747000d922a900113a8000f00b200000816000a1
:1074800061042000700520002374200081497800e9
:107490008049780082497800416d20009140780051
:1074a00000ccb30000c060002041b300d4e6b700b8
:1074b000916d20009140780000ccb30000c06000c6
:1074c0003041b300d9e6b700a16d200091407800ab
:1074d00000ccb30000c0600031c2b30001407000b6
:1074e000dae6b700616d20009140780000ccb3006f
:1074f00000c060004041b300d6e6b700716d2000c7
:107500009140780000ccb30000c060005041b3004f
:10751000d7e6b700816d20009140780000ccb30021
:1075200000c060006041b300d8e6b700b16c200035
:107530009140780000ccb30000c060007041b300ff
:10754000cbe6b700c16c20009140780000ccb300be
:1075500000c060008041b300cce6b700316c200071
:107560009140780000ccb30000c060009041b300af
:10757000c3e6b700616a20009140780000ccb300f8
:1075800000c06000c041b300a6e6b700216d200036
:107590009140780000ccb30000c060005040b300c0
:1075a000d2e6b700113a800000042000008170008c
:1075b00061042000700520002374200081497800b8
:1075c00080497800824978000000eb00200888009c
:1075d00040422f00100888004110200091407800a0
:1075e00000c3b30000c0700004e1b7008460a900cc
:1075f0009460a8000000eb008008880040422f0043
:1076000060088800011120009140780000c3b30099
:1076100000c0700010e1b70084e0a90094e0a80069
:107620000000eb009008880000e823007008880044
:107630002111200091407800f0ccb30000c0600020
:107640000044a00012e1b7008500a9009500a90040
:107650000000eb00f00888000080eb00d0088800f4
:10766000e111200091407800f0ccb30000c0600030
:1076700001c2b300014070001ee1b7008760a9009d
:107680009760a9000000eb00000988000080eb0073
:10769000e00888000112200091407800f0ccb3008f
:1076a00000c0600001c2b3000140700020e1b700db
:1076b0008780a9009780a9000000eb00800c88005b
:1076c0000000eb00900c88000000eb00b00c88007c
:1076d00010002000a00c88002119200091407800a3
:1076e00000ceb30000c06000b040b30092e1b7002c
:1076f000111920009140780030ceb30000c0600026
:107700000044a00091e1b7009081a9009381a900f5
:1077100090c1bf007040b30090e1b7000000eb00e3
:10772000d00c88000000eb00e00c88000000eb00ab
:10773000000d880010002000f00c8800c119200006
:107740009140780000ceb30000c06000b040b300ac
:107750009ce1b700b11920009140780030ceb30011
:1077600000c060000044a0009be1b7009a81a9001e
:107770009d81a9009ac1bf007040b3009ae1b70093
:107780000000eb00200d88000000eb00300d8800a9
:107790000000eb00500d880010002000400d880014
:1077a000611a20009140780000ceb30000c0600054
:1077b000b040b300a6e1b700511a20009140780014
:1077c00030ceb30000c060000044a000a5e1b700c7
:1077d000a481a900a781a900a4c1bf007040b30083
:1077e000a4e1b7000000eb00700d88000000eb0082
:1077f000800d88000000eb00a00d88000000eb0069
:10780000900d8800011b20009140780000ceb3004d
:1078100000c06000b040b300b0e1b700f11a200032
:107820009140780030ceb30000c060000044a0005a
:10783000afe1b700ae81a900b181a900aec1bf0020
:107840007040b300aee1b7000000eb00c00d88004f
:107850000000eb00d00d88000000eb00f00d880068
:107860000000eb00e00d8800a11b20009140780093
:1078700000ceb30000c06000b040b300bae1b70072
:10788000911b20009140780030ceb30000c0600012
:107890000044a000b9e1b700b881a900bb81a900ec
:1078a000b8c1bf007040b300b8e1b7000000eb0002
:1078b000100e88000000eb00200e88000000eb0096
:1078c000400e88000000eb00300e8800411c2000b4
:1078d0009140780000ceb30000c06000b040b3001b
:1078e000c4e1b700311c20009140780030ceb300d5
:1078f00000c060000044a000c3e1b700c281a9003d
:10790000c581a900c2c1bf007040b300c2e1b70089
:107910000000eb00600e88000000eb00700e880095
:107920000000eb00900e88000000eb00800e880045
:10793000e11c20009140780000ceb30000c0600040
:10794000b040b300cee1b700d11c200091407800d8
:1079500030ceb30000c060000044a000cde1b7000d
:10796000cc81a900cf81a900ccc1bf007040b30079
:10797000cce1b7000000eb00b00e88000000eb0087
:10798000c00e88000000eb00e00e88000000eb0055
:10799000d00e8800811d20009140780000ceb300f9
:1079a00000c06000b040b300d8e1b700711d2000f6
:1079b0009140780030ceb30000c060000044a000c9
:1079c000d7e1b700d681a900d981a900d6c1bf00ef
:1079d0007040b300d6e1b7000000eb00000f880054
:1079e0000000eb00100f88000000eb00300f880053
:1079f00010002000200f8800211e200091407800f8
:107a000000ceb30000c06000d040b300e2e1b70098
:107a1000111e20009140780030ceb30000c06000fd
:107a20000024a000e1e1b700e081a900e381a90002
:107a3000e0c1bf007040b300e0e1b70005e1a8007d
:107a400011e1a80013e1a8001fe1a90021e1a900ac
:107a5000c8e2a900c862a900f0e2a900d902a90001
:107a6000c802a900f102a900e202a900e222a900cd
:107a7000e242a900e262a900ca02a900e002a8004d
:107a8000e022a800e042a800e062a8007340a8003d
:107a90007360a8007380a8006740a8006760a80012
:107aa0006780a80067a0a8009660a9001f000700d3
:107ab0002d03a9002c03a90023c3bf007f40600051
:107ac00023e3b70000c0eb0024e3b70020c3bf00ee
:107ad0007f40600020e3b7005132200091407800e1
:107ae00000ceb30000c060000004a00025e3b70092
:107af0001132200091407800c0cfb30000c0600078
:107b000021e3b700213220009140780030ccb3004f
:107b100000c0600022e3b70021e3a80040a7a8004e
:107b2000f302a8000080fa00000006000000fa003e
:107b3000113a8000f00b20000081600061042000f9
:107b40007005200023742000814978008049780066
:107b500082497800616a20009140780000ccb3002f
:107b600000c06000c041b300a6e6b700216d200050
:107b70009140780000ccb30000c060005040b300da
:107b8000d2e6b700113a80000004200000817000a6
:107b900061042000700520002374200081497800d2
:107ba000804978008249780031e2a90031a2a90019
:107bb0003182a9003162a900112320009140780090
:107bc000c0cfb30000c0600031e2b70030e2a900ce
:107bd00030c2a90030a2a9003082a9003062a900f9
:107be000012320009140780090cfb30000c06000d6
:107bf00030e2b7003002a90080002000c0118800e8
:107c000033e2a90033a2a9003362a9003342a900dc
:107c100032c2bf00f043b20032e2b70032a2a90084
:107c200087e0a90097e0a90087c0a90097c0a80035
:107c300031e2a8003342a8000080fa0000000600ec
:107c40000200fa00cac2bf000044b2000004e00013
:107c500002003a006b010700020037000000eb0051
:107c60002098880060998000ff0f5000e9003600de
:107c700088c4bf00624060000004e00001003200e0
:107c8000e4003700109780000000e000060032009a
:107c9000109780009040900000c8b30000c06000c2
:107ca0000004e000db003a00208020001040780053
:107cb0000080fb00000f7800300820009e00780054
:107cc000808f50003e003200300820009e00780077
:107cd000808f50000d003c00100820009e007800ae
:107ce000808f50002f003200100820009e00780086
:107cf000808f5000c0003c00000820009e007800eb
:107d0000808f50000a003200bb003700400820007e
:107d10009e007800808f5000b7003200600820007d
:107d20009e007800808f5000b3003c008f00370029
:107d300010002000a09888000a003700a09880005a
:107d40000001e900a198800020802000e140780037
:107d5000a09e200001717800a09880000000e8003b
:107d6000a0988800a09880002180200060c0780042
:107d7000ed4f5000f1ff3a00a09880000001e900ab
:107d8000a19e2000d0c0b30000f17800a29880002e
:107d9000a19e20000040eb0000f178009f0007004a
:107da000950037004007a800cae2a80000000000c4
:107db000ca62a800000000000000fe008e0037002c
:107dc000302f2100104078000004e0001400320041
:107dd0000000eb00a098880009003700a2988000fe
:107de000a1988000a09e2000e1407800208420001f
:107df00001717800a09880000000e800a098880039
:107e0000302f2100104078000080fb000000e900c6
:107e100080007800a0988000808f5000efff3e0027
:107e2000a0988000b09888000b003700b2988000be
:107e3000b1988000a0988000808050006098200059
:107e4000e14078002084200001717800b098800023
:107e50000000e800b0988800b1988000a0032000de
:107e6000808f5000f1ff36009098800080407800ad
:107e7000d087200001487800909880004800de00fc
:107e800080407800e087200001487800e02e210043
:107e900090407800f02e21001040780000c0400093
:107ea00080407800002f21001040780000c0400082
:107eb00080407800f087200001487800e030210001
:107ec000904078000088200001487800c0302100f0
:107ed0009040780010882000014878000000eb00f6
:107ee000a09888000d003700a09880008202200032
:107ef00000014100a0988000f90040002088200087
:107f000000804000904078002084200001717800bb
:107f1000a09880000000e800a0988800a098800049
:107f2000ee0f5000f0ff3600209780000000e000c8
:107f300006003200209780009040900000c8b300f7
:107f400000c060000004e0002b003a0003c4b3004e
:107f50002284200011c0b30010c0b300c25402003c
:107f6000000000002097880023003700c081200017
:107f7000104078000080fb00c800dd00d0812000a8
:107f8000104078000080fb0000804000cf80de00c1
:107f90004f09dd00c101de00830171004f01dd00ea
:107fa00000002400010020000202400083824800fb
:107fb000e05680006101b8000400be00bc1502005c
:107fc000000000002044880031448800e081200047
:107fd000104078000080fb00c800dd00f081200028
:107fe000104078000080fb00008040004044880082
:107ff00045fc0700ee00070003c4b3002280200008
:108000008040eb0010c0b300c2540200000000002a
:10801000109788000080fa00000006000000fa00b7
:10802000312f21000040eb008048780087e0a90054
:1080300010003700da150200000000000004e00024
:10804000fcff3a00302f2100104178008280fb00b5
:10805000a09e2000614078008081fb008240e80003
:10806000302f21000148780003007800e21502005b
:1080700000000000302f2100104078008080fb00bd
:10808000a09e2000614078000004e000e9ff3a0073
:108090000080fa00000006000800fa00000f7800d7
:1080a000110798002207980033079800d0978000a6
:1080b0000000e00004003a000080eb00d097880048
:1080c0001e00900070088800d09780008000780023
:1080d0003e0090000088b9008000780070088000a1
:1080e0000080400070088800710880001e00900029
:1080f000808f5000020036000080eb00d09788008f
:10810000710880002e009000808f50000200310026
:1081100010002000d09788001e00e000040032000c
:10812000700880000000d100200f88000400370094
:1081300010002000200f88000000eb00d09788007e
:108140000080fa00000006000800fa00000f780026
:10815000110798002207980033079800d0978000f5
:108160000000e00004003a000080eb00d097880097
:108170001e00900070088800d09780008000780072
:108180003e0090000088b9008000780070088000f0
:108190000080400070088800710880001e00900078
:1081a000808f5000020036000080eb00d0978800de
:1081b000710880002e009000808f50000400310074
:1081c00010002000d097880010002000200f8800a9
:1081d0001e00e00007003200d0978000e10f400051
:1081e00004003a00700880000000d100200f8800d1
:1081f0000200370010002000200f88000080fa00e5
:10820000000006000200fa00cac2bf000044b2002b
:108210000004e00004003a00209880000000e8001c
:1082200020988800040037000000eb0020988800a8
:108230000000eb003098880021988000001020009a
:10824000808f500007003a000000eb002098880063
:10825000100020003098880010002000000f7800e7
:10826000020037000000eb00000f78001e007800cd
:108270000080fa00000006000400fa0010079800d1
:108280001e009000e25c020000000000004f780039
:1082900000000000000000001e00fb000080fa004b
:1082a000000006000400fa00000f78002147980043
:1082b0002e4090000080fb009e007800da5d0200f6
:1082c0000000000000000000000000000080fa0034
:1082d000000006000a00fa00200798003107980005
:1082e000024f98003e009000000f78000040eb0025
:1082f000204798000c0037001e007800904078005e
:108300001e0fe8002e0190002e0090000000e800f3
:108310002007980002007800e2ff07002e4090003e
:108320000040e80020479800ae4090000e489000c2
:1083300080cf5000f0ff39000080fa0000000600f6
:108340000a00fa002007980031079800024f9800b1
:108350003e009000000f78000040eb00204798009e
:108360000d003700ae0090002e0090000000e800e5
:108370002007980001007800bfff070080407800c8
:108380001e007800014878001e0fe8002e40900083
:108390000040e80020479800ae4090000e48900052
:1083a00080cf5000efff39000080fa000000060087
:1083b0000000fa0002cab30021882000a0002000bb
:1083c000c4ff07000080fa00000006000000fa0069
:1083d000a0002000a8ff07008040780070c4b30010
:1083e00080cf5000050032002188200070c4b30007
:1083f00080487800070007000400370002cab30075
:1084000021882000a0002000cdff07000080fa0096
:10841000000006000200fa00d057250001002000ed
:108420002044880031448800a00520004044880092
:108430000e007800cf0107001e007800009788002a
:10844000002e2100104078008080fb00102e2100bb
:10845000104078000080fb004800dd0000804000f4
:10846000504488000000eb00a098880015003700f9
:108470000000eb00b09888000c003700a098800046
:10848000b29880006f00b90002004000ea0040008e
:10849000208820008080400000c2b300804878001f
:1084a000b09880000000e800b0988800b098800084
:1084b000ee0f5000f1ff3600a09880000000e800a9
:1084c000a0988800a0988000e90f5000e8ff3600cf
:1084d0000080fa00000006000200fa000000eb0035
:1084e000000f78001642a8000e003700000120009f
:1084f0000100200042150200000000001e0fe800ed
:10850000400120009e0f100006003400e02e2100e4
:10851000104078008040e800e02e210001487800fb
:108520000400370016c2bf00644060000004e00091
:10853000eeff3a001662a9008a40a90018e2a900dd
:108540001942a900000a2000010020004215020083
:10855000000000000080fa00000006000400fa009d
:10856000100798001e009000a01088000000eb008b
:10857000c010880017e2a9001722a9008a40a900ac
:1085800017e2a80080108000000f7800d2ff0700db
:108590000080fa00000006000000fa0050022000ef
:1085a000eeff07000080fa00000006000200fa005b
:1085b0000000eb00000f78000000eb00c010880006
:1085c0001602a8000e003700000120000100200064
:1085d00042150200000000001e0fe800800c200081
:1085e0009e0f100006003400e02e2100104078009d
:1085f0008040e800e02e21000148780004003700a8
:108600008ac0bf00644060000004e000eeff32005a
:108610008a40a90019c2bf00644060000004e00065
:1086200009003200c1108000f0bf2f000080600000
:10863000c0108800f02e2100104078008040e80033
:10864000f02e2100014878000080fa0000000600aa
:108650000200fa000000eb00000f78001642a800ac
:108660000e0037000001200001002000421502002a
:10867000000000001e0fe800800c20009e0f10007c
:1086800006003400e02e2100104078008040e80011
:10869000e02e210001487800040037008ac0bf00a6
:1086a000644060000004e000eeff32008a40a90050
:1086b0000080fa00000006000000fa001622a80060
:1086c0008ac0bf00644060000004e000fcff32008c
:1086d0008a40a9000080fa00000006000400fa00a9
:1086e000204798002e4090000000fb00901088006a
:1086f0000000eb00000f78000e00370000012000a2
:108700000100200042150200000000001e0fe800da
:10871000800c20009e0f100006003400e02e210087
:10872000104078008040e800e02e210001487800e9
:10873000040037008ac0bf00644060000004e0000d
:10874000eeff32008a40a90018c2bf0001c8b30082
:10875000014060000004e00005003200f02e21001e
:10876000104078008040e800f02e21000148780099
:1087700019c2bf0001c8b300014060000004e0005e
:1087800005003200002f2100104078008040e800f2
:10879000002f2100014878000080fa000000060048
:1087a0000200fa000000eb00000f78001662a8003b
:1087b0000e003700000120000100200042150200d9
:1087c000000000001e0fe800800c20009e0f10002b
:1087d00006003400e02e2100104078008040e800c0
:1087e000e02e210001487800040037008ac0bf0055
:1087f000644060000004e000eeff32008a40a900ff
:1088000018c2bf000044b2000004e00005003200be
:10881000f02e2100104078008040e800f02e21006a
:1088200001487800801080000000fb000080fa0002
:10883000000006000200fa000000eb00000f7800c4
:1088400016a2a8001682a8000e0037000001200022
:108850000100200042150200000000001e0fe80089
:10886000800c20009e0f100006003400002f210015
:10887000104078008040e800002f21000148780077
:10888000040037008ac0bf00644060000004e000bc
:10889000eeff32008a40a9000080fa0000000600c6
:1088a0000200fa000000eb00000f780016a2a900f9
:1088b0001682a8000e0037000001200001002000f1
:1088c00042150200000000001e0fe800800c20008e
:1088d0009e0f100006003400002f21001040780089
:1088e0008040e800002f2100014878000400370094
:1088f0008ac0bf00644060000004e000eeff320068
:108900008a40a9000080fa00000006000200fa0078
:10891000004f780025ff07001e4078006fff07001a
:108920000080fa00000006000200fa00004f780004
:108930001147980040cbb300f4ff07001e407800b9
:1089400066ff07001e40900064ff070040ff07001d
:108950000080fa00000006000000fa000eff070089
:10896000ddfe07008040eb00e0c5b300eeff07002e
:1089700011c0b300b0c2b300ebff070011c0b300d9
:10898000c0c2b300e8ff07008040eb00d0c2b300d4
:10899000e5ff07008040eb00e0c2b300e2ff070004
:1089a00011c0b300f0c2b300dfff070011c0b30075
:1089b00000c3b300dcff070001c1b30010c3b30064
:1089c000d9ff070011c0b30020c3b300d6ff0700d2
:1089d00021c2b300b0c5b300d3ff0700f1c0b3009c
:1089e00010c4b300d0ff0700a1c0b30020c4b3007f
:1089f000cdff0700f1c0b30030c4b300caff0700c9
:108a0000a1c0b30040c4b300c7ff0700f1c0b3006a
:108a100050c4b300c4ff0700a1c0b30060c4b300da
:108a2000c1ff0700f1c0b30070c4b300beff070070
:108a3000a1c0b30080c4b300bbff0700f1c0b30006
:108a400090c4b300b8ff0700a1c0b300a0c4b30036
:108a5000b5ff0700f1c0b300b0c4b300b2ff070018
:108a6000a1c0b300c0c4b300afff0700f1c0b300a2
:108a7000d0c4b300acff0700a1c0b300e0c4b30092
:108a8000a9ff0700f1c0b300f0c4b300a6ff0700c0
:108a9000a1c0b30000c5b300a3ff0700f1c0b3003d
:108aa00010c5b300a0ff0700a1c0b30020c5b300ec
:108ab0009dff0700f1c0b30030c5b3009aff070067
:108ac000a1c0b30040c5b30097ff0700f1c0b300d9
:108ad00050c5b30094ff0700a1c0b30060c5b30048
:108ae00091ff0700f1c0b30070c5b3008eff07000f
:108af000a1c0b30080c5b3008bff070041c0b30025
:108b0000d0c5b30088ff0700c1c0b300e0c5b30003
:108b100085ff07000080fa00000006000000fa0050
:108b200040cbb30079ff07000040eb00ebfe0700ed
:108b300050cbb30075ff070019ff07000000fb00d2
:108b40009098880056ff070015ff07000000fb0003
:108b50004800dd0080007800909880000080700060
:108b60009098880033ff0700b9fe07000080fa00e4
:108b7000000006000400fa001007980080002000a2
:108b8000401988002023a8000000eb00000f7800a7
:108b9000030037001e0078000000e800000f780096
:108ba0009e007800900f2000808f5000f9ff360063
:108bb0002023a9000000eb00000f7800030037001d
:108bc0001e0078000000e800000f78009e0078008a
:108bd000900f2000808f5000f9ff360020c3bf00a7
:108be000614060000004e000fcff320000188000db
:108bf000000f78001e0090001e0878001e009000f4
:108c00000080fa00000006000000fa0042c0bf0029
:108c10007f40600001c2b3000140700042e0b70035
:108c20007e600200000000000080fa0000000600e4
:108c30000000fa000080fa00000006000000fa00c0
:108c40000080fa00000006000000fa000080fa0030
:108c5000000006000000fa00985f0200000000001b
:108c60000080fa00000006000000fa000080fa0010
:108c7000000006000000fa00d1c1b30010c0b3002c
:108c8000105402000000000003c4b3002280200042
:108c90008040eb0010c0b300c2540200000000008e
:108ca000109788000080fa00000006000000fa001b
:108cb00040998000e10f500019003a00509980005f
:108cc000e10f500016003a00d9ff07008824a900e0
:108cd0000000eb005099880000e12000004088006f
:108ce000004080000000e900004088000040800053
:108cf0000000e000faff3a009444a80080702000d1
:108d000000408800004080000000e900004088002a
:108d1000004080000000e000faff3a009444a900ff
:108d20000080fa00000006000800fa00000f78003a
:108d300011079800220798001e007800300798005d
:108d400020072000be009000808f50002c003200d1
:108d500020072000be009000808f50000a003e00d7
:108d60003e009000e20f500020003200be00900054
:108d7000e38f50001f0032003e009000e10f5000d2
:108d8000180032001e00370040072000be0090008f
:108d9000808f50001100320040072000be0090007c
:108da000808f50000900390050072000be0090005d
:108db000808f500007003200f0ff2700be009000b7
:108dc000808f50000d0032000d0037009bff070020
:108dd0000b0037008cff07000900370094ff0700e5
:108de00007003700a3ff0700050037009eff0700bc
:108df0000300370097ff07000100370092ff0700cc
:108e0000100020000080fa00000006000200fa00b6
:108e10009ec0a9000080eb00702488000080eb0059
:108e2000502488000000eb00502588000000eb0073
:108e30006025880020002000302588000000eb001d
:108e4000402588008644a900f0092000802488007d
:108e5000f0092000602488008804a8000040210058
:108e60004800de00c02488000040eb00004f78007e
:108e7000070037001e80fb00c200dd00004021001b
:108e8000008140006000b8000089be001e4fe8006d
:108e900070c0b3009e4f1000f6ff36009424a80067
:108ea0000000eb00b024880094a4a9009424a90039
:108eb0000e0037008000200050248800413221003d
:108ec0000040eb0080487800113321000040eb00a7
:108ed00080487800203321009040780060c860000e
:108ee000303321009040780060c860008ac4bf0021
:108ef000684060000004e000eeff3a00100020002f
:108f0000909a880010002000a09a88000000eb00d2
:108f1000009988000000eb00f09888000000eb004a
:108f2000509988000040eb00004f78001500370092
:108f30001e80fb0080004000a033210080804000a4
:108f40000000eb00800878001e80fb0080004000dd
:108f500060332100808040000000eb008008780032
:108f60001e81fb00c13421000040eb0000f17800bd
:108f70001e81fb00e13421000040eb0000f178008d
:108f80001e4fe80010c0b3009e4f1000e8ff3600ef
:108f900080402100d0998800d00020005025880012
:108fa0006035210010a088000140210080c0b3007e
:108fb000804878001140210040c8b3008048780004
:108fc000e13221000040eb00804878000000eb0017
:108fd000609988000080fa00000006000200fa0094
:108fe000609980000000e00015003a000000eb00ee
:108ff000a02488000000eb006024880020002000ee
:10900000302588000000eb00402588008644a90038
:10901000f009200080248800f009200060248800e6
:10902000010037009404a80094c4bf0061406000b0
:109030000004e000fbff320010002000609988006f
:1090400060998000e10f50000c003a0094c4bf000a
:109050000044b2000004e00008003a000080eb0089
:10906000502488000000eb00602488008c04a800d5
:109070008c84a800200020006099880080c4bf0074
:10908000704060000004e0000700320082c4bf00ae
:10909000704060000004e000030032000001200086
:1090a00000248800d300070088c4bf00624060002d
:1090b0000004e000020032008ec0a900a7003700c3
:1090c0008ac4bf00614060000004e0000900320073
:1090d0008cc4bf00614060000004e0000500320065
:1090e0004aff07004000200060998800100020001f
:1090f000502488008ac4bf00704060000004e00073
:10910000070032008cc4bf00704060000004e00023
:1091100003003200aa00070000012000502488004c
:109120008ac4bf00644060000004e00019003200ff
:109130008cc4bf00644060000004e0000500320001
:10914000120020008000eb0030072000944602004f
:10915000000000004000200050248800003521005d
:10916000104078000004e0000500320000352100c6
:10917000104078008040e900003521000148780067
:1091800000352100104078000004e00001003a00a2
:109190000e0307008ac4bf0001c8b300014060008d
:1091a0000004e000060032008cc4bf0001c8b30018
:1091b000014060000004e000010032006900070087
:1091c0008ac4bf00624060000004e0000d0032006d
:1091d0008cc4bf00624060000004e000090032005f
:1091e000120020008000eb00f0ff270094460200f0
:1091f000000000000080eb007024880020002000a8
:109200005024880060998000e30f500002003e0067
:109210008ec0a900510037008cc4bf0068406000b8
:109220000004e0004c0032000040eb00004f7800ea
:10923000460037008ac4bf00684060000004e000b8
:109240004500320090248000804078008034210066
:1092500001487800803421001080fb004400de00cb
:109260008040780090342100014878008000200080
:10927000502488008034210010407800684060004d
:109280000004e00013003a00903421001040780000
:109290000081fb0090342100104078008080fb00aa
:1092a000e0342100008040009040780061c0600000
:1092b0000004a200e1406000e03421000000410011
:1092c00061c16000e1cfb30010c8600010487100b8
:1092d0001200370090342100104078000081fb001c
:1092e00090342100104078008080fb00c0342100c1
:1092f000008040009040780061c060000004a2003f
:10930000e1406000c03421000000410061c1600004
:10931000e1cfb30010c86000104871009034210004
:10932000104078000004e00002003a003e00070010
:10933000050037000001eb008134210020072000e8
:1093400094460200000000001e4fe80030c0b30049
:109350009e4f1000b7ff36008ec0a9000080fa00b3
:10936000000006000000fa00aac4bf0062406000ce
:109370000004e0000e003200009a8000904090004f
:1093800000c8b30080cf500008003a00d099800098
:109390009040900040c8b30080cf500003003a00d6
:1093a000019a8000c0c8b30090409800aa24a90088
:1093b00000082000502488000080fa000000060009
:1093c0000000fa008284a8000001200050248800d8
:1093d00010002000509988000001eb008000eb0095
:1093e0005007200094460200000000000080fa00b0
:1093f000000006000000fa000000eb005099880011
:109400000001eb008000eb004007200094460200c2
:10941000000000008284a9000001200000248800d0
:109420000080fa00000006000200fa000135210069
:10943000d0c2b3008048780080342100104078000a
:109440008080fb00b0ff2f00008060000000e00083
:1094500033003a0080342100104078008080fb0007
:10946000c00f2000008060004280de004200dd006e
:10947000800078000040210000804000009a8800b1
:10948000009a8000109a88002134210020342100a5
:10949000104078000024a20080487800009a8000e4
:1094a00010409000c2c3b3008240600040c3b300cc
:1094b00080cf500018003a000040eb00004f7800c9
:1094c0000d0037001e80fb00800078006035210011
:1094d00080804000009a80001000900010407800ca
:1094e00080487800019a8000110090000000e80098
:1094f000900098001e4fe80070c0b3009e4f10000f
:10950000f0ff3600009a80006135210011009800bc
:109510000d0007000a0037004d0007000800370063
:1095200080342100104078008080fb00b0ff2f00c5
:1095300000806000e80f500001003a005f00070063
:109540000080fa00000006000000fa00413421000b
:109550000040eb00804878000000eb00e0988800b5
:109560000000eb00009988000000eb00f0988800f4
:109570000000eb00509a8800513421000040eb00bd
:1095800080487800d2998000d09980009040900067
:10959000f0c7b30000c0600010419800a133210063
:1095a000a0332100104078000024a20080487800f9
:1095b000d2998000d099800090409000f0c7b3000d
:1095c00000c0600010419800a1332100a0332100a9
:1095d000104078000024a20080487800129a800091
:1095e000109a800090409000f0c7b30000c0600067
:1095f00010419800413221000040eb008048780083
:109600000000eb0030998800113321000040eb008e
:1096100080487800203321009040780060c86000c6
:10962000303321009040780060c860007600070069
:109630000001eb008000eb003000200094460200a7
:1096400000000000f20207000080fa00000006009f
:109650000000fa005034210010407800e24f500022
:1096600002003a007903070012003700503421004d
:109670008040eb0001487800509a80000000e00034
:109680000a003a00119a800080c0b3008048780038
:10969000119a80006035210090009800119a800096
:1096a000c0c8b30090409800020037000000eb00f3
:1096b000509a88000080fa00000006000200fa00bc
:1096c000d0998000104090000080fb004600de0032
:1096d00061406000004f7800a1332100a0332100d9
:1096e000104078000024a200804878006099800033
:1096f000e80f50000c003a0080352100104078003f
:109700000080fb00b0248800b02480000000e0004e
:109710000300320000012000609988000200370039
:1097200040002000609988005034210010407800eb
:10973000e14f500016003a00d1998000e035210039
:109740009000980004030700403421001040780086
:10975000e24f500004003a00d199800040c8b300a5
:1097600090409800260037001e04e00004003a00f4
:10977000d199800080ccb300904098002000370041
:10978000d199800080c8b300904098001c00370039
:10979000103321009040780000c8b30000c0600082
:1097a0000004e00013003200403321009080fb00f1
:1097b000503321001080fb004800dd0001007000e4
:1097c0000000e00007003200403321009080fb00e1
:1097d000503321001080fb004800dd0001007000c4
:1097e0000000010011332100114078000070a10039
:1097f00080487800513421000040eb008048780018
:109800000080fa00000006000400fa006035210024
:10981000104078000046b2000004e00054003a0016
:1098200070352100104078000080fb006101b90014
:10983000028fbe00b0002000010020001e01be000b
:10984000800f5100818f590049003e001e00be006c
:10985000006001002100370022003700440037007b
:109860002000370042003700060037000b003700a9
:109870003a0037000d0037000a0037001b003700a0
:109880002b003700209980000070a00020998800ec
:10989000800020006099880035003700aa01070089
:1098a000330037006e03070031003700e03221003b
:1098b00010998800209980000000a000209988005d
:1098c0006132210010c0b3008048780020998000e8
:1098d0000070a0002099880025003700e5010700ee
:1098e000230037002400070021003700a0352100a5
:1098f000104078000080fb0080007800e0332100f9
:109900000080400010998800209980000000a0008d
:10991000209988006132210010c0b300804878008f
:10992000209980000070a000209988001000370066
:10993000209980000070a00020998800a0352100a7
:10994000104078000081fb008035210090407800b5
:10995000e033210001717800050037000001eb00c1
:109960008000eb0020002000944602000000000070
:109970000080fa00000006000600fa008035210091
:1099800010407800e14f500011003a00603521008e
:10999000104078007f4060000004e0000c003a00b6
:1099a000209980000070a000209988007035210067
:1099b00010407800e34f500003003a0010002000f0
:1099c00040998800020037000000eb0040998800b1
:1099d00080352100104078000004e000f9003a00d2
:1099e00060352100104078007f406000e24f500059
:1099f000f4003a00a0352100104078006f4060006c
:109a00000004e000ef003200a03521009040780013
:109a10006fc060000080fb00e10f5000e9003c00d7
:109a20006199800000022000808f5000e5003a001c
:109a3000209980000070a00020998800a0352100a6
:109a40009040780000c8b30000c060000004e0004f
:109a500011003a00a0352100904078006fc06000ee
:109a60000080fb0080004000603321000080400047
:109a70001000780010079800a03521009040780071
:109a80006fc060008080fb00e034210061407800fe
:109a90004047980010003700a03521009040780022
:109aa0006fc060000080fb0080004000a0332100f8
:109ab000008040001000780010079800a0352100b9
:109ac000904078006fc060008080fb00c0342100af
:109ad00061407800404798004e409000614060002f
:109ae0000004e00007003a000e81e8000e80e80064
:109af00090407800b0cfb30000c06000004978000b
:109b0000050037008e80e8000e80e80010407800e5
:109b10000024a00080487800a03521009040780003
:109b200000c8b30000c060000004e0000b003a0071
:109b3000a0352100904078006fc060008080fb005d
:109b40001e009000000178008180400060332100f9
:109b500000804000020878000a003700a03521008c
:109b6000904078006fc060008080fb001e00900075
:109b70000001780081804000a03321000080400077
:109b8000020878007035210010407800e34f500043
:109b900022003a001e00900090007800000028008b
:109ba000008060000000e00015003200a0352100b8
:109bb0009040780000c8b30000c060000004e000de
:109bc00008003a00a0352100904078006fc0600086
:109bd0008080fb00e0342100008040001014a000d1
:109be00007003700a0352100904078006fc060006a
:109bf0008080fb00c0342100008040001014a000d1
:109c00001e0190001e0090009040900040c8b300dc
:109c100000c07000104198006a0037008e80e80094
:109c20000e80e800104078000024a20080487800f0
:109c30001e00900090007800000028000080600066
:109c40000000e000120032001e0190001e00900093
:109c500090409000f0c7b30000c060001041980031
:109c60001e0190001e0090009040900000c4b300c0
:109c700000c07000104198009e009000220020005b
:109c8000500020009446020000000000060037004b
:109c90001e0190001e0090009040900000c4b30090
:109ca00000c07000104198008e80e8000e80e8002f
:109cb000104078000024a200804878004e409000b8
:109cc000624060000004e00006003a001e009000c0
:109cd0009000780000002800008060000000e00094
:109ce00023003200a03521009040780000c8b30066
:109cf00000c060000004e00009003a00a035210027
:109d0000904078006fc060008080fb00e03421004c
:109d100080804000d0cfb300914860000800370039
:109d2000a0352100904078006fc060008080fb006b
:109d3000c034210080804000d0cfb3009148600043
:109d40001e0190001e00900090409000b0c3b30030
:109d500000c06000104198009e009000220020008a
:109d6000500020009446020000000000060037006a
:109d70001e0190001e00900090409000b0c3b30000
:109d800000c0600010419800a0352100904078008c
:109d90006fc060000080fb00000040008000780081
:109da000a04a200000804000000f78001e007800cc
:109db00090407800d0cfb30080c060001e007800d3
:109dc000014878000080fa00000006000000fa0058
:109dd000909a80000000e0002c003a001000200063
:109de000909a8800a09a80000000e00027003a00c6
:109df00010002000a09a8800503421001040780004
:109e0000e24f500007003a00d19980000040eb007b
:109e100080487800d199800080ccb30090409800b1
:109e20001a0037005034210010407800e14f5000f4
:109e300016003a000000eb00509a8800019a80005a
:109e400080c0b30080487800019a8000603521000e
:109e500090009800019a800040c8b300904098009c
:109e600010002000509a8800119a800080c0b30032
:109e700080487800119a8000603521009000980099
:109e8000119a800000c8b300904098000080fa004a
:109e9000000006000000fa000000eb0000998800b6
:109ea0000000eb00f098880050342100104078004a
:109eb000e24f50000a003a00119a800080c0b300bf
:109ec00080487800119a8000e035210090009800c9
:109ed000119a800080ccb3009040980018003700a1
:109ee000c03521009080fb00d03521001080fb00a0
:109ef0004800dd000100700080007800309980008b
:109f0000808f500007003100c03521009080fb0099
:109f1000d03521001080fb004800dd0001007000fa
:109f2000309988000c010700d1998000e0352100ac
:109f300090009800d199800080ccb30090409800a8
:109f40000080fa00000006000200fa0060352100df
:109f50009040780000c8b30080cf500043003a0022
:109f60004132210000ccb3008048780090352100b8
:109f7000104078000080fb00000f78001e00780081
:109f8000e20f50000c0032001e007800e30f50007a
:109f90001d0032001e007800e10f50000100320069
:109fa0002f003700c06c2900109988002001200084
:109fb000309988002d00370080352100104078004e
:109fc0000080fb000000400080007800a07829009d
:109fd00000804000100078001099880010998000df
:109fe0000080e8009040780060322100014878004d
:109ff000109980006300400090407800703221008a
:10a0000001487800190037008035210010407800a1
:10a01000e24f50000e003e008035210010407800d5
:10a020000080fb000000400080007800c07829001c
:10a03000008040001000780010998800109980007e
:10a04000104078000080fb0030998800070037003e
:10a05000413221000040eb008048780003003700c7
:10a06000413221000040eb00804878000080fa0077
:10a07000000006000400fa00e13521000040eb007a
:10a0800080487800f13521000040eb0080487800de
:10a0900060352100904078007fc060000080fb00a8
:10a0a000100798001e009000e10f50001a003200c7
:10a0b0009e009000e28f50001b0032001e009000b6
:10a0c0000000e000010032004200370020998000cb
:10a0d0000070a00020998800e03521001040780031
:10a0e000804078000104a000e0352100014878009c
:10a0f00040998000e10f500036003a00e035210021
:10a1000010407800804078000114a000e035210064
:10a11000014878002f003700209980000070a000cf
:10a12000209988002b003700209980000070a00043
:10a1300020998800a03521009040780000c8b30025
:10a1400000c060000004e0000a003a00a0352100d1
:10a15000904078006fc060000080fb0080004000ed
:10a16000603321000080400010007800000f78006c
:10a1700009003700a0352100904078006fc06000d2
:10a180000080fb0080004000a033210000804000e0
:10a1900010007800000f78001e0078009000780012
:10a1a00000002800008060000000e000090032008c
:10a1b0001e007800900078000040200000806000c1
:10a1c0000000e00003003200e135210010c0b300c0
:10a1d000804878002099800001082000010060007c
:10a1e0000000e00008003200e035210010998800ee
:10a1f000209980000000a000209988006132210091
:10a2000020c0b300804878000080fa0000000600fb
:10a210000000fa0094a4a900209980000108200001
:10a22000010060000000e0001f003a001033210030
:10a230009040780000c8b30000c060000004e00057
:10a240000c0032005034210021c0b30001487800d6
:10a25000f09880000000e00001003a000dff0700c8
:10a260000000eb00a09a88000000eb00909a8800a4
:10a2700037003700119a800080c0b3008048780012
:10a28000119a80006035210090009800119a80009a
:10a29000c0c8b30090409800d199800040c8b30076
:10a2a000904098002a0037006035210090407800e7
:10a2b00000c8b30000c060000004e00010003200dd
:10a2c0005034210011c0b30001487800009980008b
:10a2d0000000e00001003a00eefe07000000eb0085
:10a2e000a09a88000000eb00909a8800e098800017
:10a2f0000000e00016003a00b4fe0700140037002a
:10a300005134210020c0b30080487800119a8000a9
:10a3100080c0b30080487800119a80006035210029
:10a3200090009800119a800040c8b30090409800b7
:10a330000000eb00a09a88000000eb00909a8800d3
:10a34000e09880000000e00001003a009ffe070056
:10a350000080fa00000006000200fa0080c0b3008e
:10a36000004f780030998000e70f500011003e0048
:10a3700030998000004f7800403421001040780070
:10a380000004e00004003a004134210010c0b30092
:10a3900080487800070037004034210010407800e2
:10a3a000e14f500003003a004134210020c0b300c7
:10a3b00080487800319980001e80fb0000805000aa
:10a3c00030998800d09980001e487800e03521003f
:10a3d000309a880020998000610060000000e00051
:10a3e00016003a0009003700319a80001299800067
:10a3f00012407800804878000100e800309a880018
:10a400000200e800109988001e4fe9001e04e000d9
:10a41000f5ff3a000b003700319a80001299800056
:10a4200012407800804878000100e800309a8800e7
:10a430000200e800109988001e4fe9001e04e000a9
:10a44000f5ff3a000080fa00000006000200fa0062
:10a45000009a800090407800114798001e409000bc
:10a460000081fb00203321009080fb00303321006d
:10a470001080fb004800dd0001007000800f5100db
:10a4800007003600203321009080fb00303321008c
:10a490001080fb004800dd000100700010479800ac
:10a4a000203321009080fb00303321001080fb001e
:10a4b0004800dd0001007000800078001e40900020
:10a4c0000080fb0000815000f00f20008000610040
:10a4d000203321009041780060c8610010c87000ee
:10a4e000c810de0030332100104178006048610060
:10a4f00010c870000040eb00004f780018003700d3
:10a50000f03221009080fb00003321001080fb001e
:10a510004800dd0001007000000178009e80fb0013
:10a52000e035210061407800004978000201e80030
:10a53000f00f200080006100f0322100904178008f
:10a5400060c8610010c87000c810de000033210030
:10a55000104178006048610010c870001e4fe8008c
:10a560001e4090009e4f1000e5ff3900203321006f
:10a570009080fb00303321001080fb004800dd009c
:10a58000010070000000e00013003200119a80000a
:10a5900080c0b30080487800119a8000e035210027
:10a5a00090009800009a8000104090000044b20093
:10a5b0000004e00004003a00119a800080ccb3004f
:10a5c0009040980024003700119a800080c8b300a2
:10a5d0009040980020003700119a800080c0b3009e
:10a5e00080487800119a8000603521009000980022
:10a5f000119a800040c8b300904098004033210079
:10a600009080fb00503321001080fb004800dd00eb
:10a61000010070000000e00007003200403321001c
:10a620009080fb00503321001080fb004800dd00cb
:10a6300001007000000001001033210090407800fc
:10a640000170a10001487800e09880000000e0005f
:10a6500001003a00ddfd07000080fa00000006005e
:10a660000200fa00209980000070a0002099880064
:10a670000000eb00602588000040eb00004f7800f0
:10a68000070037001e80fb00c200dd0000402100f3
:10a69000008140006000b8000089be001e4fe80045
:10a6a00070c0b3009e4f1000f6ff36009424a8003f
:10a6b0000040eb00004f7800090037001e81fb00ce
:10a6c000c13421000040eb0000f178001e81fb0046
:10a6d000e13421000040eb0000f178001e4fe8005b
:10a6e00010c0b3009e4f1000f4ff3600e13321008c
:10a6f0000040eb00804878009424a90080402100ad
:10a70000d099880000402100009a8800009a8000bb
:10a71000109a88008035210090407800e0322100b6
:10a7200001487800e0322100104078000004e00089
:10a7300003003a00000120006099880007003700fc
:10a7400012002000e1322100100020009446020097
:10a750000000000000022000609988000080fa00dc
:10a76000000006000400fa002047980031479800d6
:10a7700000402100000f78002e4090000080fb0078
:10a7800000004000800078003e4090000080fb0008
:10a79000008040004300dd001e0f40009e00780056
:10a7a000114090000074a100904098003e4090003d
:10a7b0000004e00007003a002e4090000080fb00fb
:10a7c0008000400060332100008040001e087800b7
:10a7d000060037002e4090000080fb008000400003
:10a7e000a0332100008040001e0878001e01780080
:10a7f00092409000f0cbb30000c060001041980080
:10a800001e007800640140009240900000c4b30034
:10a8100000c07000104198000080fa00000006009f
:10a820000400fa0020479800314798003e4090000d
:10a830000080fb004300de00610060000004e000d7
:10a84000030032008040eb002e409000c5ff07005f
:10a850003e4090000080fb004200de00610060008e
:10a860000004e0000300320011c0b3002e4090004d
:10a87000bcff07002e4090000080fb00000040005d
:10a8800080007800a04a200000804000000f78007f
:10a890001e007800be409000014878000080fa0059
:10a8a000000006000400fa00204798003147980095
:10a8b0002e4090000004e0000d003a00119a800044
:10a8c00080c0b30080487800119a80006035210074
:10a8d00090009800119a8000c0c8b3009040980082
:10a8e000d199800040c8b300904098002300370001
:10a8f0002e4090000080fb000000400080007800a7
:10a900003e4090000080fb00008040004300dd00de
:10a91000800078000040210000804000000f780097
:10a920001e0078009040900040c8b30080c07000c6
:10a930001e007800114098002e4090000080fb001f
:10a9400000004000800078003e4090000080fb0046
:10a95000008040004300dd0080007800404021007e
:10a96000008f40001e0078009040900040c8b30067
:10a9700080c070001e007800114098000080fa002e
:10a98000000006000a00fa002047980031479800ae
:10a9900022079800634798003e4090000004e000c2
:10a9a000070032002e4090000080fb008000400035
:10a9b000a033210000804000100f7800060037000f
:10a9c0002e4090000080fb0080004000603321009a
:10a9d00000804000100f78001e00e00003003a00e5
:10a9e0000000eb0040079800390037002e0090006f
:10a9f000800078001e007800110098001e0078008a
:10aa0000ee409000014878001e0078001040900051
:10aa100002c4b300824060001e007800114098001c
:10aa20001e0078009040900080c8b30080c0700085
:10aa30001e007800114098003e4090000004e000a5
:10aa4000110032002e4090000080fb00000040000a
:10aa500080007800a03321000080400000017800d1
:10aa60002e4090000080fb00000040008000780035
:10aa7000a033210000804000104078000024a20094
:10aa800000497800100037002e4090000080fb0045
:10aa9000000040008000780060332100008040000a
:10aaa000000178002e4090000080fb000000400074
:10aab0008000780060332100008040001040780062
:10aac0000024a200004978001e007800400798008a
:10aad0004e0090000080fa00000006000600fa0018
:10aae000004f780094c4bf000042b2000004e000b0
:10aaf0005f0032001e80fb0080004000a033210078
:10ab000000804000100378001e80fb0080004000a1
:10ab1000a033210000804000100078001000be002b
:10ab20000204200003002000000278008102780067
:10ab3000020078008300780000016200018062005a
:10ab40006102b80014079800250798001e009000c5
:10ab5000ae009000c000dd0000002000100798004b
:10ab6000210798001e009000ae0090006112b8000e
:10ab700014079800250798001e019000ae01900070
:10ab80000200700083807000008bbe001e80fb00fe
:10ab900080004000a03321000080400010027800b7
:10aba0001e80fb0080004000a03321000080400098
:10abb000100078001001be000004200001002000f9
:10abc0000000690081806900008abe001e80fb00d1
:10abd0000000400080007800a03321000080400089
:10abe000000178001e80fb0000004000800078001b
:10abf000a033210000804000104078000024a20013
:10ac0000004978001e80fb0080004000a033210036
:10ac100000804000100178001e80fb008000400092
:10ac2000a033210000804000100078001040900008
:10ac30000044b200104198001e80fb0080004000dc
:10ac4000a033210000804000100178001e80fb002e
:10ac500080004000a03321000080400010007800f8
:10ac60009040900000c4b30000c0680010419800fc
:10ac70000080fa00000006000600fa0042c0bf0093
:10ac80000080fb004500de000080fb0020079800ec
:10ac90009002800010079800ff3ffc002104200074
:10aca0009140780000ceb30000c0700042e0b700d1
:10acb0001e00900090028800066102000000000063
:10acc00090028000000f7800ff3ffc002e009000f3
:10acd00067406000c500dd0042c0bf007f406000eb
:10ace0000140700042e0b7001e007800900288002a
:10acf0000080fa00000006000c00fa00604798008f
:10ad000071479800024f980032c0bf000080fb00de
:10ad1000000f780002802100030020006e409000a8
:10ad20008080fb0000c020000088b90001002000e6
:10ad300002014000838148007e4090000080fb00bb
:10ad40004a00dd000100200002004000838048002e
:10ad50004008de000100200032e0b7000080210042
:10ad600001002000000178006e4090000080fb0090
:10ad70006300b900800078007e4090000080fb00f6
:10ad8000008040004a00dd000000410020079800dc
:10ad90002e009000fe60020000000000804078005d
:10ada00000c0eb0000c06000304798000e489000e3
:10adb0000080fb00500798005e009000f30f5000e9
:10adc0000d0032005e009000f40f500010003200c1
:10add0005e009000f20f50000100320012003700b8
:10ade0003e4090000080fb00640060004280de0076
:10adf000204798000e0037003e4090000080fb0086
:10ae0000680060004380de0020479800080037009b
:10ae10003e4090000080fb00700060004480de0037
:10ae200020479800020037000040eb0020479800c0
:10ae30001e00780032e0b7002e4090000080fb003a
:10ae40000080fa00000006000600fa004047980063
:10ae50005147980032c0bf000080fb00000f78000f
:10ae600002802100030020004e4090008080fb0003
:10ae700000c020000088b90001002000020140004d
:10ae8000838148005e4090000080fb004a00dd00a6
:10ae90000100200002004000838048004008de00de
:10aea0000100200032e0b70020042400003b8800ad
:10aeb0000080210001002000000178004e40900039
:10aec0000080fb006300b900800078005e409000c5
:10aed0000080fb00008040004a00dd0000004100cf
:10aee000100798009e0090001e009000286102004c
:10aef0000000000060ff07001e00780032e0b7008d
:10af00000080fa00000006000c00fa00204f9800b4
:10af10000000eb004007980032c0bf000080fb003b
:10af2000000f78000000eb003007980003003700a6
:10af30003e0090000000e800300798003e009000be
:10af4000e20f500007003c003e0090008040780077
:10af500032c1b3002e48900067ff0700e10f500098
:10af6000f3ff320002802100030020002e489000f1
:10af70008080fb0000c020000088b9000100200094
:10af800002014000838148003e0090004a00dd003d
:10af90000100200002004000838048004008de00dd
:10afa0000100200032e0b7000080210001002000f5
:10afb000000178002e4890000080fb006300b9007b
:10afc000800078003e009000008040004a00dd00d4
:10afd00000004100100798004e0090000080e8003b
:10afe000400798001e0090000080e80010079800bd
:10aff0001e009000fe60020000000000804078000b
:10b0000000c0eb0000c0600040479800ce009000f8
:10b01000f03f2000808f500003003c004e40900025
:10b02000e14f4000ecff3a00ce00900000402000cd
:10b03000808f500002003a000000eb0040079800ab
:10b040001e00780032e0b7004e0090000080fa0049
:10b05000000006001600fa00881f780020579800ac
:10b0600032c0bf000080fb00600798000000eb00ca
:10b07000000f9800030037000e0890000000e80061
:10b08000000f98000e089000e20f500007003c00ef
:10b090000e0890008040780032c1b3002e5090001e
:10b0a00015ff0700e10f5000f3ff32000e0890007b
:10b0b000e30f500008003a006e00900032e0b70045
:10b0c000709b80000030a000709b88003000200042
:10b0d000200f9800810137000e0890000000e80062
:10b0e000700798007e009000e30f500017003a00b0
:10b0f0000000eb0070079800140037007e009000fd
:10b100000000e800700798007e009000e30f5000f8
:10b1100002003a000000eb0070079800fe0090006b
:10b120000e089000808f500008003a006e009000da
:10b1300032e0b700709b80000010a000709b880078
:10b1400010002000200f9800640137007e0090005e
:10b150008040780042c1b3002e509000e6fe070008
:10b160000000e000e5ff3200028021000300200023
:10b170002e5090008080fb0000c020000088b900a5
:10b180000100200002014000838148007e00900001
:10b190004a00dd00010020000200400083804800da
:10b1a0004008de000100200032e0b70000802100ee
:10b1b00001002000000178002e5090000080fb006c
:10b1c0006300b900800078007e009000008040009d
:10b1d0004a00dd0000004100400798002e5090001a
:10b1e00049ff07000000e00003003200709b800070
:10b1f0000020a000709b8800e0362100104f7800ee
:10b20000709b80000000a100709b88000000eb0094
:10b210003007980010002400003b8800ce0090000a
:10b220000080eb002861020000000000ce009000ca
:10b23000f00f200020610200000000004e0090008e
:10b240000080e800400798000040eb00404798006d
:10b250003e0090000000e800300798003a003700f8
:10b260002e5090008080fb00f00f20000088b90075
:10b27000800078004e4090000080fb00008040007d
:10b28000d001070010079800709b800061006000eb
:10b290000000e00004003200709b80000000a1006c
:10b2a000709b88000f0037001e009000ce009000b9
:10b2b00028610200000000004e4090000080fb006a
:10b2c000ce00900020610200000000004e009000bf
:10b2d0000080e800400798003e0090000000e80071
:10b2e000300798004e4090000040e800404798002a
:10b2f0000e003700ce0090000080eb0028610200b5
:10b3000000000000ce009000f00f2000206102003d
:10b31000000000004e0090000080e8004007980008
:10b320003e0090000000e800300798004e4090007a
:10b33000e14f400004003a00be009000f0032000fe
:10b34000808f5000ebff34004e409000e14f4000f2
:10b3500004003200be009000f0032000808f5000f7
:10b36000bfff340044fe07000000eb0030079800e8
:10b370004e409000e14f4000f3ff3a00e0362100dc
:10b380001e48780002802100030020002e5090000b
:10b390008080fb0000c020000088b9000100200070
:10b3a00002014000838148007e0090004a00dd00d9
:10b3b0000100200002004000838048004008de00b9
:10b3c0000100200032e0b7000080210001002000d1
:10b3d000000178002e5090000080fb006300b9004f
:10b3e000800078007e009000008040004a00dd0070
:10b3f000000041000080e80040079800ce00900067
:10b400004e0090000000e80040079800010078001e
:10b41000fe6002000000000040479800ce0090004f
:10b420004e0090000000e8004007980001007800fe
:10b43000026102000000000010079800250037009c
:10b440002e5090008080fb00f00f20000088b90093
:10b45000800078004e4090000080fb00008040009b
:10b4600058010700800078001e009000808f500077
:10b47000080032006e00900032e0b700709b800040
:10b480000070a000709b880070002000200f9800c2
:10b4900092003700ce0090004e0090000000e800bf
:10b4a0004007980001007800fe60020000000000e4
:10b4b00040479800ce0090004e0090000000e80049
:10b4c00040079800010078000261020000000000bf
:10b4d000100798004e409000e14f4000d8ff3a001e
:10b4e0000080210001002000000178002e50900013
:10b4f0000080fb006300b900800078000e08900017
:10b50000008040004a00dd00000041005007980024
:10b510000080210001002000000178002e509000e2
:10b520000080fb006300b900800078007e0090007e
:10b53000008040004a00dd00000041004007980004
:10b5400002802100030020002e5090008080fb002c
:10b5500000c020000088b900010020000201400066
:10b56000838148000e0890004a00dd0001002000a1
:10b5700002004000838048004008de0001002000f7
:10b5800032e0b7005e00900002610200000000009f
:10b59000100798005e009000fe60020000000000ae
:10b5a000404798007e0090000000e00003003a0051
:10b5b0001e0090000000e800100798001e00900098
:10b5c000e30f500007003600709b80000010a000c1
:10b5d000709b8800f1ceb3004e40900001406000a7
:10b5e0004047980002802100030020002e50900068
:10b5f0008080fb0000c020000088b900010020000e
:10b6000002014000838148007e0090004a00dd0076
:10b610000100200002004000838048004008de0056
:10b620000100200032e0b7004e4090000080fb0097
:10b63000ce00900020610200000000001e0090007b
:10b64000ce009000286102000000000030002400bd
:10b65000003b880088fd07004e4090000084fb00fe
:10b660004e009000fe60020000000000800f5400b9
:10b6700007003a004e009000026102000000000046
:10b68000800078001e009000808f5000080032007b
:10b690006e00900032e0b700709b80000070a00048
:10b6a000709b880070002000200f98000b0037006e
:10b6b0000e089000804078002e509000e2fd0700b8
:10b6c0006e00900032e0b700709b80000000d10057
:10b6d000614060000080fb00200f98002e08900061
:10b6e0004f0478000080fa00000006000e00fa0007
:10b6f00032c0bf000080fb0040079800008021009e
:10b70000010020004008de000100200032e0b70008
:10b710000040eb00004f7800a20037000040eb0033
:10b72000304f98000040eb00204f98000000eb00e5
:10b73000100798000000eb00300798000300370066
:10b740003e0090000000e800300798003e009000a6
:10b75000e20f500007003e003e009000804078005d
:10b7600042c1b3001e40780063fd07000000e00006
:10b77000f3ff32003e009000e30f500008003a0053
:10b780004e00900032e0b700709b80000010a000d7
:10b79000709b88001000200060079800860037002a
:10b7a0000000eb00300798000d0037003e009000cd
:10b7b0008040780032c1b3001e4078004efd070083
:10b7c0000000e00003003a003e4890000040e8001e
:10b7d000304f98003e0090000000e80030079800cd
:10b7e0003e009000e20f5000f0ff36003e4890000f
:10b7f0000004e00024003a008040eb001e40780086
:10b8000091fd070002802100030020009e80fb00c4
:10b8100000c020000088b9000100200002004000a4
:10b82000838048004008de000100200032e0b700bd
:10b830000080210001002000000178009e80fb00b4
:10b8400000c020000088b9000000410020079800d7
:10b8500030002400003b8800ae0090000000eb00a8
:10b860002861020000000000ae009000300f2000b0
:10b870002061020000000000fffc07004e00900065
:10b8800032e0b700460037003e489000e14f5000dc
:10b8900003003a004e00900032e0b700400037004d
:10b8a0003e489000e24f500035003a0032c1b300ec
:10b8b00021c0b3001e4078000ffd07000000e0002b
:10b8c0000b003a0032c1b3008040eb001e4078000c
:10b8d00009fd07000000e00005003a0020002000fc
:10b8e000300798000040eb00204f98001800370008
:10b8f0000000eb0030079800030037003e00900086
:10b900000000e800300798003e009000804078007a
:10b9100032c1b3001e407800f7fc0700e10f500071
:10b9200003003a003e009000e20f5000f3ff3600a3
:10b930003e0090000040e800204f98002e48900004
:10b94000e34f500002003a000040eb00204f980007
:10b95000ae4890001e4078003bfd07001e40780076
:10b9600069fd07000000e00002003a001e40780078
:10b97000b8fd07004e00900032e0b7000800370025
:10b980004e00900032e0b700709b80000060a00085
:10b99000709b880060002000600798000600370058
:10b9a0001e4fe80010c0b3009e4f10005bff360032
:10b9b0000000eb00600798006e0090000080fa0025
:10b9c000000006001000fa0060079800ee009000ea
:10b9d000d01f2000808f500006003600709b800032
:10b9e0000050a000709b88000080eb00700798005a
:10b9f0006d0037006e009000f20f2000110009006a
:10ba00000280d800004f780032c0bf000080fb00e9
:10ba1000500798000000eb00400798000300370033
:10ba20004e0090000000e800400798004e00900093
:10ba3000e20f500007003e004e009000804078006a
:10ba400032c1b3001e407800abfc0700e10f50008c
:10ba5000f3ff32004e009000e30f500008003a0060
:10ba60005e00900032e0b700709b80000060a00094
:10ba7000709b88000080eb00700798004a00370038
:10ba800002802100030020009e80fb0000c02000f7
:10ba90000088b900010020000201400083814800b5
:10baa0004e0090004a00dd0001002000020040002e
:10bab000838048004008de000100200032e0b7002b
:10bac0000080210001002000000178009e80fb0022
:10bad00000c020000088b900800041004e009000a6
:10bae0004a00dd0000804000e03fb00030079800d1
:10baf00000202000100798003e009000fe60020029
:10bb000000000000200798003e0090000080e9003f
:10bb1000300798001e0090000000e9001007980010
:10bb20001e0090000000e000090032006e0090004e
:10bb3000f20f2000110009000280d8008000fd00f3
:10bb4000800078002e009000808f5000eaff3a00bd
:10bb50001e0090000000e00008003a00709b80008a
:10bb60000000a000709b88005e00900032e0b700eb
:10bb70000080eb00700798000b0037003e0090003b
:10bb80000080e800300798003e009000026102004b
:10bb900000000000200798005e00900032e0b7002f
:10bba0002e009000700798007e0090000080fa0040
:10bbb000000006001400fa0070079800010f9800ba
:10bbc0008e089000d01f2000808f500006003600a5
:10bbd000709b80000050a000709b880050002000e7
:10bbe000100f9800cf0037000e089000f20f2000d1
:10bbf000110009000280d800000f780032c0bf0099
:10bc00000080fb005007980030002400003b8800b3
:10bc10000000eb0040079800030037004e00900042
:10bc20000000e800400798004e009000e20f50002e
:10bc300007003c004e009000804078001e00780015
:10bc400032c1b3002cfc0700e10f5000f3ff3200bb
:10bc50004e009000e30f500008003a005e00900094
:10bc600032e0b700709b80000060a000709b8800ed
:10bc700061002000110f9800aa0037000280210007
:10bc8000030020009e00780000c020000088b9005a
:10bc90000100200002014000838148004e00900016
:10bca0004a00dd00010020000200400083804800bf
:10bcb0004008de000100200032e0b70000802100d3
:10bcc00001002000000178001e0078006300b90028
:10bcd000800078004e009000008040004a00dd00a7
:10bce0000000410030079800e036210090407800c5
:10bcf000214798000e08900032ff0700800078006e
:10bd00007e009000808f50000c003a00709b8000f5
:10bd1000610060000000e00008003a005e00900052
:10bd200032e0b700e0362100ae40900001487800d4
:10bd30000000eb00100f98007a003700e036210079
:10bd4000ae409000014878001e0078006efc0700ad
:10bd5000200798002e0090000000e00008003a0044
:10bd60005e00900032e0b700709b80000040a000b1
:10bd7000709b880040002000100f98006900370079
:10bd8000be0090002e009000008040003007980018
:10bd90007e009000be0090002861020000000000bc
:10bda0000e089000f20f2000110009000280d80058
:10bdb0008000fd00be009000206102000000000035
:10bdc000adfb070000000000000000003e009000f6
:10bdd00002610200000000008040780000c0eb001b
:10bde00000c06000404f98004e4890000081fb006a
:10bdf000fe009000f00f200000806000800f5100d6
:10be0000080032005e00900032e0b700709b8000b6
:10be10000070a000709b880071002000110f980036
:10be2000400037003e009000fe600200000000006d
:10be30008040780000c0eb0000c06000404f9800d8
:10be40004e4890008080fb000e089000f20f20000a
:10be5000811f7800110009000280d80000017800dd
:10be600001007800cf007800808f50000800320079
:10be70005e00900032e0b700709b80000070a00070
:10be8000709b880070002000100f9800250037007c
:10be90003e0090000000e800300798003e0090004f
:10bea00002610200000000004880de00804078004f
:10beb00000c0eb0000c06000404f98004e4890006a
:10bec0000081fb007e009000c800de00f00f200023
:10bed00000806000800f5100080032005e0090007a
:10bee00032e0b700709b80000070a000709b88005b
:10bef00071002000110f98000a003700ae0090007a
:10bf0000e03f2000808f500002003a001e007800c1
:10bf100050fc07005e00900032e0b7000000eb002c
:10bf2000100f98001e0890000080fa000000060024
:10bf30000400fa0060352100104078007f40600066
:10bf4000e14f50006b003a00a0352100104078000e
:10bf50000004e00067003a007035210010407800ce
:10bf6000e64f500025003a0090352100104078003f
:10bf70000080fb0010079800100220009e00900037
:10bf8000808f500005003200200220001e0190002a
:10bf9000800f51000e00320018003700e0322100ff
:10bfa00010407800e14f500014003a00e06d290085
:10bfb000720040001099880090002000309988009d
:10bfc0004132210000ccb300804878000b003700dc
:10bfd000e032210010407800e14f500007003a00a5
:10bfe000e076290010998800c0012000309988006f
:10bff0004132210000ccb300804878006035210038
:10c000001040780002c6b3008240600000c2b30056
:10c0100080cf500037003a00703521001040780082
:10c020000080fb00000f78001e007800e30f500036
:10c03000210032009e007800e38f500007003c0092
:10c040001e017800e10f51002a0032001e00780026
:10c05000e20f500008003200260037009e007800f2
:10c06000ea8f50000c0032001e017800eb0f5100e7
:10c07000190032001f003700c036210010998800d7
:10c0800010002000309988004132210010ccb3000c
:10c0900080487800170037004132210000c8b30003
:10c0a000804878009035210090407800c03621000b
:10c0b000014878000f003700d03621001099880021
:10c0c00010002000309988004132210010c8b300d0
:10c0d00080487800070037004132210000c8b300d3
:10c0e000804878008035210090407800d0362100cb
:10c0f000014878000080fa00000006000a00fa00fb
:10c1000042c0bf0001ceb300014060000004e00067
:10c1100003003a000000eb004007980034003700ad
:10c12000f10c20009140780080cfb30000c0600087
:10c130000004a000cfe0b700812480003107980000
:10c1400060248000200798001124800011079800c7
:10c150009ec0bf000080fb004600de006140600022
:10c16000004f78000000eb00802488000000eb0006
:10c17000602488000000eb00102488008ec0a90015
:10c180008284a80000012000002488009ec0a8002e
:10c190000040fe00f10c20009140780080cfb300f9
:10c1a00000c06000cfe0b7009e40780061c0600032
:10c1b000614060004601dd00e10920009140780007
:10c1c000f0cbb30000c06000024070009ee0b700fa
:10c1d0003e00900080248800ae009000612488001a
:10c1e0001e009000102488001100200041079800d4
:0cc1f0004e0090000080fa0000000600e5
:020000040000fa
:102f24001c1300005000000000000000001400000a
:102f340020000000000000006c13000002000000ec
:102f4400000000006e1300000200000000000000fa
:102f5400e21200003a00000002000000000000003d
:102f6400000100000000000000000000000000005c
:102f740064000000000000000000000000000000e9
:102f8400000000000000000000000000000000003d
:102f94000000000005030000020000000000000023
:102fa4000000000081000a0000000000000800008a
:0c2fb400e20a0000000000000000000025
:020000040000fa
:10c1fc001080ba00000006001000ba000000060013
:10c20c00801f78000500fc0050052000303b8800a2
:10c21c00a00a2000303b880061e7a8000000000065
:10c22c000000000061e7af00feff37004f00780010
:10c23c00000006008088bb000000060080c8bb0020
:10c24c00000006008008bb00000006008048bb0010
:04c25c0000000600d8
:020000040000fa
:082fc0000040da000000fe00f1
:00000001FF
